:10000000020A05908002EEF0A3EFF0908002E0FE7D
:10001000A3E0FF908344EEF0A3EFF0908344E0FE72
:07002000A3E04E70F622324E
:10002B00020BF7C2AFC2D3C2D4E4F58E75C870F51C
:10003B0093759401759502F5C9F5F875F901F5A855
:10004B00F5B8F59AF5A9F5B953C9FD2275F9014330
:06005B00BC1E53BD04228F
:0300630002002672
:10006B00020B4290821E120261908221EDF0E09011
:10007B008224F0908222E0FEA3E0FF908344EEF016
:10008B00A3EFF0908344E0FEA3E04E604E90832BF1
:10009B00E0FF90832AE0C39FFF908221E0FEEFC335
:1000AB009E40E0908224E0FF14F0EF602B90832BB6
:1000BB00E0242AF582E43482F583E0FF90821E125D
:1000CB000241EF12014990821FE475F00112017D8C
:1000DB0090832BE004F080CB7F01227F0022E49001
:1000EB00832AF0A3F02212002E120C2D22FFFF44C4
:1000FB0057494E5435020A4CBB010689828A83E06C
:10010B00225002E722BBFE02E32289828A83E49318
:10011B0022BB010CE58229F582E5833AF583E022C7
:10012B005006E92582F8E622BBFE06E92582F8E2B5
:10013B0022E58229F582E5833AF583E49322BB011C
:10014B000689828A83F0225002F722BBFE01F3223A
:10015B00F8BB010DE58229F582E5833AF583E8F0DA
:10016B00225006E92582C8F622BBFE05E92582C886
:10017B00F222C5F0F8A3E028F0C5F0F8E58215826D
:10018B0070021583E038F022BB0110E58229F5825D
:10019B00E5833AF583E0F5F0A3E0225009E92582E7
:1001AB00F886F008E622BBFE0AE92582F8E2F5F0B4
:1001BB0008E222E5832AF583E993F5F0A3E993227C
:1001CB00F8BB0111E58229F582E5833AF583E8F066
:1001DB00E5F0A3F0225009E92582C8F608A6F02223
:1001EB00BBFE09E92582C8F2E5F008F222E0FCA388
:1001FB00E0FDA3E0FEA3E0FF22ECF0A3EDF0A3EE05
:10020B00F0A3EFF022A8828583F0D083D082120274
:10021B0027120227120227120227E473E493A3C5C5
:10022B0083C5F0C583C8C582C8F0A3C583C5F0C517
:10023B0083C8C582C822E0FBA3E0FAA3E0F922F849
:10024B00E0FBA3A3E0F925F0F0E58215827002151F
:10025B0083E0FA38F022EBF0A3EAF0A3E9F022E70F
:10026B0009F608DFFA807BE9D39850F3E92FF9E818
:10027B002FF819E718F6DFFA8068E709F208DFFABA
:10028B00806080E388828C83E709F0A3DFFA8052D9
:10029B00E309F608DFFA804AE9D398500EE92FF903
:1002AB00E82FF819E318F2DFFA8037E309F208DFD9
:1002BB00FA802F88828C83E309F0A3DFFA802389ED
:1002CB00828A83E0A3F608DFFA801789828A83E4A7
:1002DB0093A3F208DFF9800A89828A83E0A3F208EC
:1002EB00DFFA02037C80B180F980A580C680DC80B8
:1002FB00F180738010808380E98087808780D9802C
:10030B00E180BC8073D3E998EA9C5039E92FF582E0
:10031B00EA3BF583E82FF8EC3BFC0582D58202150E
:10032B00831582E493C8C582C8CCC583CC0582D51E
:10033B00820215831582F0C8C582C8CCC583CCDF79
:10034B00D9DED7802E89828A83ECFAE493A3C8C5C1
:10035B0082C8CCC583CCF0A3C8C582C8CCC583CC1E
:10036B00DFE9DEE7800D89828A83E493A3F608DF59
:10037B00F9ECFAA9F0EDFB22D3E998EA9C5038E9A5
:10038B002FF582EA3BF583E82FF8EC3BFC0582D591
:10039B00820215831582E0C8C582C8CCC583CC0503
:1003AB0082D5820215831582F0C8C582C8CCC5835D
:1003BB00CCDFDADED880BC89828A83ECFAE0A3C872
:1003CB00C582C8CCC583CCF0A3C8C582C8CCC583B5
:1003DB00CCDFEADEE8809C809888F08E83EF6001AA
:1003EB000E4E608DED2402B404005085F582EB2493
:1003FB0002B4040050E123234582AB83239002F027
:10040B0073908113EFF0A3ECF0A3EDF0A3EAF0A34C
:10041B00EBF0908113E090811BF0908114E0FEA330
:10042B00E0FF908118120241781C7C817D01120340
:10043B00E47B017A81791B908114E0FEA3E0240117
:10044B00FDE43EFC12094990821BEEF0A3EFF09005
:10045B00821BE0A3E0FF908114E0FCA3E0241CF5D9
:10046B008274813CF583EFF090821BE0FEA3E0EEFB
:10047B00FF908114E0FCA3E0241DF58274813CF510
:10048B0083EFF01200E97B017A81791B908114E0F4
:10049B00A3E02403FD120A917B017A81791B780872
:1004AB00E6FE08E6FF908222EEF0A3EFF07D051248
:1004BB00006E90821DEFF0E070037FFD2290821D95
:1004CB00E0C3648094805003E0FF2290811BE0FF27
:1004DB00908113E06F60037FFC2290811CE030E77A
:1004EB001A7B017A81791B7D057C00120949EF4E3D
:1004FB0060037FFA2290811DE0FF227B017A8179D4
:10050B0020908116E0A3E024FEFD7808E6FE08E6C5
:10051B00FF908222EEF0A3EFF012006E90821DEF9F
:10052B00F0E070037FFD2290821DE0C36480948015
:10053B005003E0FF227B017A81791B908116E0FE4C
:10054B00A3E02403FDE43EFC120949EF4E60037F58
:10055B00FA22908116E0FEA3E0FF7B017A81791CE1
:10056B00C003C002C001A3120241A801AC02AD033B
:10057B00D001D002D0031203E47F0022908002EE60
:10058B00F0A3EFF0A3120261908002E0A3E054010C
:10059B00908009F0908002E0FEA3E0FFEEC313FE13
:1005AB00EF13FF908002EEF0A3EFF0E4F5F19080F3
:1005BB0002E0FEA3E0EEF5F2908002E0A3E0F5F39B
:1005CB0075F40175F88F30FCFD908009E0603C906C
:1005DB008007E0FEA3E0D39400EE9400402D75F865
:1005EB0083908004E475F00112024A120103F5FCBA
:1005FB00908004E475F00112024A120103F5FDD25A
:10060B00FE90800774FFF5F012017D75F88F9080D6
:10061B0007E0FEA3E0C39402EE9400404B908004ED
:10062B00E475F00112024A120103F5FA908004E41A
:10063B0075F00112024A120103F5FB908004E47578
:10064B00F00112024A120103F5FC908004E475F0EC
:10065B000112024A120103F5FDD2FE90800774FFCE
:10066B0075F0FE12017D80A6908007E0FEA3E04EA0
:10067B00602375F88C908004E475F00112024A1225
:10068B000103F5FA908004E475F00112024A12019D
:10069B0003F5FBD2FEE4F5F8221200F112005778B5
:1006AB00087600087607120C43908338120210006C
:1006BB000002BCC291C292C293C294E4908336F002
:1006CB00A2A233908001F07B017A83792C90800673
:1006DB001202617B0A7D007C017F30120BBE90837E
:1006EB0037EFF0E0703690832CE030E004D291804D
:1006FB0002C29190832CE030E104D2938002C2932A
:10070B0090832CE030E604D2928002C29290832C2C
:10071B00E030E704D2948011C294800D908337E0CF
:10072B00FFE4FCFDFEA31202047F0A7E001200030D
:10073B007B017A8379409080061202610B7D107CDD
:10074B00007F10120B85908337EFF0E070117B0167
:10075B007A837940120AEF90833C120204800A904C
:10076B00833C120210000000007B017A83793C90DD
:10077B008007E4F0A37402F07F007E501205877FA0
:10078B00E87E031200030206D222908009EFF0A349
:10079B00EDF0A3EAF0A3EBF0A3E06005D3947D406A
:1007AB00037FFF2290800E120241EA494B70037FB8
:1007BB00FF2290800AE0908011F090800BE0FEA366
:1007CB00E0EE908012F090800BA3E0908013F0E4A9
:1007DB00A3F090800DE0908015F090800D75F002E5
:1007EB00A42402FBE435F0FAC002C003908009E0B8
:1007FB00FF7B017A807911908118120261D003D0AE
:10080B00027D057C0012040C908111EFF0E0600278
:10081B00FF22E4908112F090800DE0FF908112E0B6
:10082B00C39F5043E025E02413F582E43480F58325
:10083B00E0FE908112E025E02414F582E43480F58B
:10084B0083E0FDEEEDFF90800E120241908112E0ED
:10085B0075F002A4F58285F083EE8FF01201CB9038
:10086B008112E004F080B07F0022908009EFF0A3AA
:10087B00EDF0A3EAF0A3EBF0A3E06009D394D074FE
:10088B0080948740037FFF2290800E120241EA4939
:10089B004B70037FFF2290800AE0908011F09080D4
:1008AB000BE0FEA3E0EE908012F090800BA3E090A3
:1008BB008013F090800DE0E4908014F090800DE0B8
:1008CB00908015F090800D5407600BE0FF1313130D
:1008DB00541F04F0800B90800DE0FF131313541F73
:1008EB00F0908009E0FF90800DE02402FBE433FAE6
:1008FB00C002C0037B017A807911908118120261CA
:10090B00D003D0027D057C0012040C908111EFF016
:10091B00E06002FF2290800DE0FF7E007B017A8079
:10092B007913C003C002C001A3120241A801AC029B
:10093B00AD03D001D002D0031203E47F00229082DA
:10094B001E120261908221ECF0A3EDF074FFA3F074
:10095B00A3F090821E1202419082251202617B004D
:10096B007A007900C003C002C001908225120241B7
:10097B00D082D083D0E06B7008E965827003EA65A2
:10098B0083606EE4908228F0A3F0908221E0FEA3B6
:10099B00E0FF908228E0FCA3E0C39FEC9E505290B6
:1009AB008225E475F00112024A120103FF908223A3
:1009BB00E0FCA3E0FDECEF6D25E0FFE433FE747C7F
:1009CB002FF582740C3EF583E493FC740193FD9038
:1009DB008223E0FEA3E0EEFFECFEEF6DFF9082239F
:1009EB00EEF0A3EFF0908228E475F00112017D8008
:1009FB0099908223E0FEA3E0FF22787FE4F6D8FDF6
:100A0B00758109020A4C0206A4E493A3F8E493A3AC
:100A1B004003F68001F208DFF48029E493A3F85435
:100A2B0007240CC8C333C4540F4420C8834004F4B8
:100A3B0056800146F6DFE4800B01020408102040CB
:100A4B0080900C59E47E019360BCA3FF543F30E5CA
:100A5B0009541FFEE493A360010ECF54C025E06040
:100A6B00A840B8E493A3FAE493A3F8E493A3C8C50E
:100A7B0082C8CAC583CAF0A3C8C582C8CAC583CAFF
:100A8B00DFE9DEE780BE90821E120261908221EDCB
:100A9B00F07B007A007900C003C002C00190821E77
:100AAB00120241D082D083D0E06B7008E96582706E
:100ABB0003EA6583602D908221E06027D2819082CA
:100ACB0021E0FF14F0EF601990821E120241120117
:100ADB0003FF120C6B90821FE475F00112017D80F5
:100AEB00DDC28122908002120261908002120241CB
:100AFB009080051202619080051202411201039051
:100B0B00800BF090800512024190000112011C90A5
:100B1B00800AF090800512024190000212011C9095
:100B2B008009F090800512024190000312011C9085
:100B3B008008F01201F822C0E0C083C082C0D075DB
:100B4B00D000C007908000E4F0C2AFE5AB30E01DF1
:100B5B00E5ADF0E0FF90832AE0242AF582E43482AD
:100B6B00F583EFF090832AE004F053ABFED2AFD0C5
:100B7B0007D0D0D082D083D0E032908002EFF0A3A8
:100B8B00ECF0A3EDF0A3EBF0908002E0FFA3E0FA12
:100B9B00A3E0FBC002C003A3E090800DF0908006A1
:100BAB0012024190800E120261D003D0027D03121B
:100BBB00079522908002EFF0A3ECF0A3EDF0A3EBEE
:100BCB00F0908002E0FFA3E0FAA3E0FBC002C003B9
:100BDB00A3E090800DF090800612024190800E12DF
:100BEB000261D003D0027D0212087522C0E0C0F072
:100BFB00C083C082C0D075D000C000C006C2C690F2
:100C0B008344E0FEA3E04E600A90834474FFF5F04A
:100C1B0012017DD006D000D0D0D082D083D0F0D0BE
:100C2B00E03275C870E4F5CDF5CC75CBBC75CACD8B
:100C3B0043A820D2C8D2AF2243B70275A78075ABA9
:100C4B0080E4F5AE75AFE0D2BDC281D2AF22428354
:100C5B0044000041832A0041832B00020800070057
:100C6B00908222EFF0E0F5ACE5A730E0FB53A7FE56
:100C7B00220000C0C1C1810140C30103C00280C278
:100C8B0041C60106C00780C7410500C5C1C4810428
:100C9B0040CC010CC00D80CD410F00CFC1CE810ED9
:100CAB00400A00CAC1CB810B40C90109C00880C8EA
:100CBB0041D80118C01980D9411B00DBC1DA811A58
:100CCB00401E00DEC1DF811F40DD011DC01C80DC2A
:100CDB00411400D4C1D5811540D70117C01680D659
:100CEB0041D20112C01380D3411100D1C1D0811068
:100CFB0040F00130C03180F1413300F3C1F2813259
:100D0B00403600F6C1F7813740F50135C03480F429
:100D1B00413C00FCC1FD813D40FF013FC03E80FED8
:100D2B0041FA013AC03B80FB413900F9C1F88138E7
:100D3B00402800E8C1E9812940EB012BC02A80EA59
:100D4B0041EE012EC02F80EF412D00EDC1EC812C27
:100D5B0040E40124C02580E5412700E7C1E6812658
:100D6B00402200E2C1E3812340E10121C02080E069
:100D7B0041A00160C06180A1416300A3C1A2816257
:100D8B00406600A6C1A7816740A50165C06480A429
:100D9B00416C00ACC1AD816D40AF016FC06E80AED8
:100DAB0041AA016AC06B80AB416900A9C1A88168E7
:100DBB00407800B8C1B9817940BB017BC07A80BA59
:100DCB0041BE017EC07F80BF417D00BDC1BC817C27
:100DDB0040B40174C07580B5417700B7C1B6817658
:100DEB00407200B2C1B3817340B10171C07080B069
:100DFB0041500090C191815140930153C052809258
:100E0B0041960156C057809741550095C194815426
:100E1B00409C015CC05D809D415F009FC19E815ED7
:100E2B00405A009AC19B815B40990159C0588098E8
:100E3B0041880148C0498089414B008BC18A814A56
:100E4B00404E008EC18F814F408D014DC04C808C28
:100E5B0041440084C185814540870147C046808657
:100E6B0041820142C043808341410081C180814066
:010E7B004036
:00000001FF
